:1000000000308A003C280000831A0A28A500030E4D
:10001000A6000F288312A500030EA600A6140A0846
:10002000AD008A018313A50E0408A7002008A800CC
:100030002108A9002208AA002308AB002408AC006C
:1000400083128C308400001C27280C1842282708B3
:1000500084002808A0002908A1002A08A2002B0873
:10006000A3002C08A4002D088A00260E830083120A
:10007000250EA61883160900FF2383169000003072
:100080008A00292A36088F0035088E0083168515C8
:100090008312851D6128BF0ABF1B60283F08013CF1
:1000A000031860280130BF00BD00400B58286028AD
:1000B0000130C000BE01B701B801B901BA01BB00EF
:1000C0006B28BF033F08803A7E3C031C6B28FF303F
:1000D000BF00BD01C001BE0A3E08073C03188628C8
:1000E000BA0A0130BB003A083B3C03188528BA0124
:1000F000B90A39083B3C03188528B901B80A380801
:10010000173C03188528B801B70ABE010130BC00AE
:100110000C108A11272849308400000803199F28F1
:100120000130A100A001A00B9328A10B92284A3016
:10013000A000A00B992800000000800B90287C2ACA
:10014000CA01CB01CC01CD01490DA000A00DFC30AE
:10015000A0051F08C33920049F000330A000A00B96
:10016000AF28CE019F149F18B32883161E08831250
:10017000CF004F0DA2001E0DA300A20DA30DFC3059
:10018000A2052208CA0723080318230FCB07003053
:1001900003180130CC07003003180130CD074E089A
:1001A0007F3C031CD528CE0AB228CD0CCC0CCB0C3E
:1001B000CA0CCD0CCC0CCB0CCA0CCD0CCC0CCB0C83
:1001C000CA0CCD0CCC0CCB0CCA0CCD0CCC0CCB0C73
:1001D000CA0CCD0CCC0CCB0CCA0CCD0CCC0CCB0C63
:1001E000CA0C0130CD054A08A1004B08A20000341A
:1001F000C901A0202208C2002108C1000130C900A5
:10020000A0202208C4002108C3000230C900A02099
:100210002208C6002108C5000330C900A02022081A
:10022000C8002108C7000034831685128312851682
:100230000830A100000000000000A1172E29A11322
:10024000D10C03188512031C851621172E292113A2
:10025000A10B202900000000000085121C30840042
:10026000840B3029A11B1F29211B272900340408D6
:10027000D0004A0EF038CC00CC07E23ECD00323E32
:10028000CF004A080F39CD07CD07CF07E93ECE0092
:10029000CE07CE07490E0F39CE07CF07CE0DCF0DB3
:1002A000CF09CF0D49080F39CF07CC0D0730CB0050
:1002B0000A30CF07CE03031C5929CE07CD03031CF8
:1002C0005D29CD07CC03031C6129CC07CB03031C9C
:1002D00065294B3084000730500584074F300402F5
:1002E00003198E290008A000031D7C29501A8C29AF
:1002F000D0197E2920307F290830D0003030A00767
:10030000CA010408C9002008CB002008D10014212C
:10031000490884004B08A000840A6E290008A00048
:100320003030A0072008D100142100344C08A1016E
:100330004B0203189E294B08A000AA29A0010830EF
:10034000CD00CB0DA00D4C0820020318A000A10D7C
:10035000CD0BA129003421084908CB006430CC0022
:1003600096212008C90021083030031DBE294A18F3
:10037000C429CA19C4294A1A2030C029CA114A12EC
:10038000A1072108D10014214908CB000A30CC0074
:1003900096212008C90021083030031DD329CA192D
:1003A000D7294A1A2030A1072108D1001421303062
:1003B000C9074908D100142100343708C900183092
:1003C000CA00AB212E30D10014213808C9000130F9
:1003D000CA00AB213A30D10014213908C9000130DC
:1003E000CA00AB213A30D10014213A08C9000130CB
:1003F000CA00AB212C30D1001421093084004208FE
:10040000CA004108C90037212C30D100142109301D
:1004100084004408CA004308C90037212C30D100A9
:100420001421093084004608CA004508C900372154
:100430002C30D1001421093084004808CA00470834
:10044000C90037210D30D10014210A30D100142108
:10045000DF2A84011F3083051F1383161F149F1486
:100460001F159F15073083129F0083168512831274
:100470008512AE010130AF00B001B101B201B3018C
:10048000B4012030B500C330B600B701B801B901DE
:10049000BA01BB01BC01BE01BF01FF30C000073083
:1004A00099008316050803308312A000A00B562A7A
:1004B00019088C118316990183121F1383161F14B8
:1004C0009F141F159F111F169F161F1383129F172E
:1004D0001F141F3065000000000000000000000035
:1004E000B5309000C2308F00F7308E0083160C14A8
:1004F00008308312C9008B2883169B019C131C149F
:100500001A088312B300013083169B009C131C143D
:100510001A088312B4003308B5070318B60A340862
:10052000B5020030031C0130B602F8208316851591
:100530008312BD018519BD0AC0308B04BC080319A4
:10054000E12AF820BD08031DDB2A0A30C9002D303E
:10055000D1001421C90BA72A2C30D1001421093055
:1005600084004208CA004108C90037212C30D1005C
:100570001421093084004408CA004308C900372107
:100580002C30D1001421093084004608CA004508E7
:10059000C90037212C30D1001421093084004808CB
:1005A000CA004708C90037210D30D10014210A3094
:1005B000D1001421E02ABB080319E02ADD29BB0180
:0605C000BC019E2A63004D
:0442000000000000BA
:104220004300500046002D004C004F00470047005F
:104230004500520020005600650072002E0020004C
:0A42400030002E00380034000000AA
:10426000280043002900200064006A0070006100FB
:1042700072006B0040006100730074007300620004
:104280002E0069006E0066006F00200032003000D2
:06429000300034000000C4
:1042A00054006F002000620065002000750073005C
:1042B00065006400200066007200650065006C0007
:1042C0007900200062007900200043005000460081
:1042D00020006D0065006D006200650072007300D3
:0242E0000000DC
:02400E008439F3
:00000001FF
